:10000000112411E0A0E0B1E0EEE5FDE002C00590B2
:100010000D92AA30B107D9F711E001C01D92A53C9D
:10002000B107E1F763C500001895000018950F921D
:100030000FB60F9305B1007E05B90BB10C7E0BB95D
:10004000002700930B010F910FBE0F901895000031
:1000500000000000000000000000000000000000A0
:100060000000000098C108C200000000000000006D
:100070007894DDCF78940FC10000000000000000EC
:1000800000000000729A18955C9A1895F69972987B
:10009000F7995C98189540414445464760630403CE
:1000A00007042C035400550020004300680065003D
:1000B0006D006E00690074007A002C00200045007D
:1000C0006E00610073002B005A0066004D002C0387
:1000D00053005400530020004D0075006C00740064
:1000E000690070006C00650078003A00200047004D
:1000F0006100730062006F007800300368006500E3
:10010000680061004000680072007A002E007400F0
:1001100075002D006300680065006D006E006900C9
:1001200074007A002E006400650016034E0065001E
:1001300075006500720020005700650072007400B1
:1001400010034900730074007700650072007400AA
:10015000280341006B00740069007600650072009E
:10016000200044002F0041002D00570061006E0068
:1001700064006C0065007200120353006F006C0095
:100180006C0077006500720074002C034400690065
:1001900067006900740061006C0065007200200057
:1001A0006E0070006E002D00410075007300670046
:1001B00061006E006700000009022900010100C013
:1001C00032090400000203000000092110010001AF
:1001D00022A2000705810340000A07050203400030
:1001E0000A1201000200000040C016DF05000101F4
:1001F00002030106A0FF0903A101850425010921CD
:1002000015002780841E0075209501B10209222661
:10021000FF0075089505B1A205018505093B253E3E
:10022000750895018102093A26FF00953E82020178
:100230008506093B253E95019102093A26FF009566
:100240003E920201C00600FF0903A10185031500CB
:1002500025017501950809087908B102850109048D
:100260007904B1A227C0FF00007510090579056760
:1002700021D1F000550D468813B1A28502250175E4
:100280000109067906B10227C0FF000075100907B1
:100290007907B102C0001F920F920FB60F9211247E
:1002A0002F933F934F935F936F937F938F939F937E
:1002B000EF93FF9360910D01462F062E000C550B16
:1002C0002091780030917900FA01EE0FFF1FE15F75
:1002D000FE4F80819181280F391F31832083FA01DD
:1002E0003296E770FF27EA56FF4FE491E0937C00D7
:1002F00070910C01CA0101967F33A9F4FC01EE0F45
:10030000FF1FEF54FE4F3183208321E030E001C016
:10031000220F6A95EAF73091B201232B2093B201A4
:10032000452B09F4189A87709927009731F420918A
:100330000C012F5F2F7320930C0180930D01FF910F
:10034000EF919F918F917F916F915F914F913F912D
:100350002F910F900FBE0F901F90189580910B0159
:1003600095B1282F2F71907E922B95B92BB190E0EB
:10037000AC0133E0559547953A95E1F7407155E06A
:10038000959587955A95E1F78370842B922F9C7EE3
:10039000892B8BB908951F920F920FB60F921124DB
:1003A0002F933F934F935F938F939F93EF93FF937D
:1003B0002091CE00789480910701382F307287FF0A
:1003C0000AC0332309F446C04D9B44C090910801F4
:1003D000906890930801482F407486FF1CC080915C
:1003E000600105B402FE04C0A89A16BC95E095BD54
:1003F0008E335CF4E82F082E000CFF0BE15AFE4F01
:1004000022838F5F8093600107C090910801906400
:100410009093080101C080E0332339F08C33ECF471
:10042000411102C04D9919C05E982091090199B1FE
:10043000422F022E000C550B892F90E09595879541
:100440008427952784FF0BC080E1822781608093F9
:10045000090105C02093CE00BECF5E9AE6CFFF9182
:10046000EF919F918F915F914F913F912F910F90BD
:100470000FBE0F901F9018951F920F920FB60F92FC
:1004800011248F939F93EF93FF9388E98093C90082
:10049000789480910E01909120018917CCF490916D
:1004A000070192FF06C04E9B04C09068909307011D
:1004B0000FC0E82F082E000CFF0BE15EFE4F92816B
:1004C0009093CE008F5F80930E0188EB8093C900DC
:1004D000FF91EF919F918F910F900FBE0F901F9002
:1004E0001895823023E09207D1F044F4853021E062
:1004F0009207A1F18130934049F00895833023E0C1
:10050000920791F084309340A9F0089562E170E081
:1005100081EB91E00E94C2031092B201089562E162
:1005200070E08FE991E004C062E070E08AE091E061
:100530000C94C20389B18695807190910901907FD6
:10054000892B809309016AE070E080E091E00E94CD
:10055000C2031092080110920901089560E470E04E
:100560008FE591E00E94C2031092600108958230ED
:1005700023E0920781F02CF48630924009F4B9C050
:100580000895833023E0920709F48AC084309340B1
:1005900009F48EC0089562E170E08FE991E00E9455
:1005A000F6038091A1019091A2019093890080931C
:1005B00088008091A3019091A40190938B00809377
:1005C0008A008091A5019091A60190938D0080935F
:1005D0008C008091A7019091A8019093990080933D
:1005E00098008091A9019091AA0176E0969587954F
:1005F0007A95E1F79093BF008093CF008091AB0193
:100600009091AC01E6E096958795EA95E1F7909395
:10061000BF008093D2008091AD019091AE019C010A
:100620002095309530939B0020939A002091AF0144
:100630003091B001A9014095509550939D00409391
:100640009C004091A0014EBBF69B07C06A9A089798
:1006500050F080917100846004C06A9880917100AC
:100660008B7F80937100F79B08C0549A2830310526
:1006700050F080917100886004C05498809171009E
:10068000877F809371008EB3807C21F08091710010
:10069000816003C0809171008E7F80937100089506
:1006A00062E070E08AE091E00E94F6030C94AE01F3
:1006B0006AE070E080E091E00E94F6032091010181
:1006C000309102014091030150910401DA01C90106
:1006D000B695A79597958795BC01CD01605C7D4B3C
:1006E000804F9F4F0E9475063093CD002093CC0021
:1006F000089560E470E08FE191E00E94F60380913C
:100700002001882329F010920E0188EB8093C90004
:1007100008958091E800982F9570D9F3847008951A
:1007200021E02093E9002091E80020FD10C020EA9C
:100730002093E800FC018091E80085FF04C08191CE
:100740008093F100F8CF1092E80081E0089580E0F6
:10075000089522E02093E9002091E80022FF10C0D4
:1007600020EA2093E800FC018091E80085FF04C0A6
:100770008091F1008193F8CF1092E80081E0089514
:1007800080E00895FF920F931F93CF93DF938C0126
:100790008091C3019091C401EB01861797070CF477
:1007A000EC018EEFF82E0E948903811119C0C1342B
:1007B000D10514F49C2F01C090E4F801192E26FCF9
:1007C000059026FE01900092F1001A94C1F78F0166
:1007D000C91BD109F092E800209729F7903419F34A
:1007E000DF91CF911F910F91FF900895CB01089554
:1007F000CF93DF938091DA0080FF28C01092DA0057
:100800008091D90080FF14C0589A81E08093D7006E
:1008100081EB8093D80082E189BD09B400FEFDCF51
:1008200081E98093D8001092E0001092E1000DC0A1
:100830005C985998589881E18093D80080E189BDEF
:100840001092D70081E08093E100212C8091E1009B
:1008500091E09093E10083FF0EC01092E9001092A6
:10086000EC0022E32093ED009093EB0094E0909352
:10087000E800212C5C9880FF0AC059989091D8001C
:1008800095FD05C090EB9093D80090E199BD84FF51
:100890000DC0599A8091D80085FF08C082E189BDBA
:1008A00009B400FEFDCF80E98093D8001092E900E2
:1008B0003091E80033FF17C19091F1008091F10071
:1008C000C091F1002091F100863019F440E4420F0C
:1008D00002C040E3480F4093CE00D091F100409118
:1008E000F1004091F1006091F100337F3093E80016
:1008F00050E0562B5093C4014093C301913209F448
:1009000077C040F4913009F44FC098F0923009F468
:100910004FC0E6C0913809F49AC020F4903809F429
:1009200071C0DEC0923809F4BAC0913A09F4CCC063
:10093000D7C0833049F018F4813031F0D1C0853010
:1009400039F0893079F0CCC0C13009F0C9C0B8C0E5
:100950008EEF8093E8000E9489038C2F806880933B
:10096000E300C1C0C23008F0BBC08EEF8093E80046
:100970002C2E5C98CC23B1F05C9A81E08093E90046
:100980008093EB0091EC9093EC0096E39093ED0054
:1009900022E02093E9008093EB0080EC8093EC0050
:1009A0009093ED008EE71FC08B3009F099C088C08E
:1009B000813019F0833009F093C0C11191C0DF7705
:1009C000D33008F08DC09EEF9093E800D093E900FB
:1009D00081FD86C089E18093EB0081E090E001C059
:1009E000880FDA95EAF78093EA001092EA007BC05C
:1009F000813009F075C08C2F90E0922BDF91CF9160
:100A00000C94B702863049F0883009F43AC081115D
:100A100067C00E94890381E04FC0822D8064282E28
:100A2000223009F1233031F0213009F059C081EE34
:100A300091E016C0C93008F053C08EE990E0CC2395
:100A400079F0FC012491820F911DC150F8CF8630BE
:100A5000F9F4F22DF0642F2E213249F48AEC91E062
:100A6000FC01649109C088EB91E069E205C0223283
:100A7000B9F583EF91E062EA70E0DF91CF910C94D9
:100A8000C2030E948903822D81708093F10018C0F7
:100A90008A3031F5D23020F50E9489030FC08111D0
:100AA0001FC00E948903D093E9008091EB0085FB71
:100AB000882780F91092E9008093F1001092F100EC
:100AC0008EEF8093E8000FC0813051F4822D8F7B30
:100AD000282E8C2F90E0922BDF91CF910C947102F5
:100AE00081E28093EB00DF91CF91089580E885BF8C
:100AF00014BE98E1909360001092600080936100B2
:100B00001092610081E083BF94E8909364009FEFAE
:100B100094B990EC97B99BEB9AB994E49EB993EF92
:100B200090937E0080937F00629B04C06A9A80E469
:100B30008093A001729880E480937C008FEF809373
:100B40007A0081E480937C008BE180BF81E0809318
:100B5000B10182E080939F0183E080930A0180E0ED
:100B600090E00E94A706843041F44AE050E060E043
:100B700070E080E091E00E94970685E080935F013D
:100B800086E080931F0188E98093C90020910101CC
:100B9000309102014091030150910401DA01C90131
:100BA000B695A79597958795BC01CD01605C7D4B67
:100BB000804F9F4F0E9475063093CD002093CC004C
:100BC0008FEF9FEF9093970080939600909387000C
:100BD000809386008AEA809390008093800089E168
:100BE000809391008093810083E08093BF008FEF1A
:100BF0008093D10082E88093C00087E08093C10099
:100C000089E88093C20080E48093C40081E38093EC
:100C1000D80012E004E078E0D72EE8EBCE2E2C9836
:100C20008091E10080FD02C081E201C080E3F89480
:100C30008093E2001093E9000093F0001092E90025
:100C4000D092F00078948895F8941092F000109368
:100C5000E9001092F00078941092E2002C9A0E9421
:100C6000F8038091C90085FD0EC08FE191E00E94DC
:100C7000A903882341F080912001882321F010925C
:100C80000E01C092C90080916001893214F4A89BC2
:100C900010C0C091C9008C2F8F778093C9008FE559
:100CA00091E00E94900381111092600115BCC093E5
:100CB000C900F999B4CF80E0E82E81E0F82EC0E0B9
:100CC000D0E0CE010E94A706F70191917F0189171C
:100CD00031F090BDF894FA9A7894F99AA0CF2196C1
:100CE000F0E0CA30DF0769F79ACFA1E21A2EAA1BFB
:100CF000BB1BFD010DC0AA1FBB1FEE1FFF1FA217CC
:100D0000B307E407F50720F0A21BB30BE40BF50BC8
:100D1000661F771F881F991F1A9469F76095709551
:100D2000809590959B01AC01BD01CF010895DC0138
:100D3000CB01FC01F999FECF06C0F2BDE1BDF89AE6
:100D4000319600B40D9241505040B8F70895F9998A
:0E0D5000FECF92BD81BDF89A992780B5089517
:0A0D5E0004802500000320C00000FF
:00000001FF
